:020000020000FC
:020000005BC0E3
:0200080007C02F
:1000160050C022BB1895789400E205BF88950895D4
:1000260033E0F9DF3A95E9F708953FE1F4DF3A95D1
:10003600E9F708952066EFDF2F79F2DF2066EBDF20
:100046002F79EEDF08952066EBDF2F79E4DF206657
:10005600E7DF2F79E0DF08952066DDDF2F79E0DF27
:100066002066DEDF2F79D7DF08952066D4DF2F796B
:10007600DCDF0895DADFCFDF0895D7DFD6DFD5DFFF
:10008600D4DF0895FADF4A95E9F70895D3DFE4DF70
:10009600DADFD9DFD8DFE0DFD6DFD5DFD4DFCADFAE
:1000A600C9DFC8DFE2DF0895F1DFF0DFEFDFEEDF63
:1000B6000895F8940FED0DBF00E007BB0FEF08BBE6
:1000C6000FEF01BB00E002BB20E000E808B900E04A
:1000D6000FBD00E00DBD0CBD04E00BBD07EB0ABD76
:1000E60009E00EBD00E409BF00E00BBF5CC000E6FE
:1000F60002BBFDCFD9DFD8DFD7DFD6DF00C006B31E
:100106000C7F0C5FE1F742E0BDDF06B30C7F0C5FAE
:10011600B1F700E009BF00E20BBF00E20ABF0CEF37
:1001260000BD789400E705BF8895BEDFBDDFBCDF64
:10013600BBDF4FEFA7DF4FEFA5DF4FEFA3DF44E6AF
:10014600A1DFB2DFB1DFB0DFAFDFD9CFADDFACDF2C
:10015600ABDFAADF4FEF96DFA7DFA6DFA5DFA4DFC1
:1001660047E390DFA1DFA0DF9FDF9EDFC8CF9CDFE4
:100176009BDF9ADF99DF48E285DF96DF95DF94DF24
:1001860093DF47E37FDF90DF8FDF8EDF8DDFB7CF33
:100196008BDF8ADF89DF88DF45EA74DF85DF84DF6E
:1001A60083DF82DFACCF789446E06CDFB79BDFCF8E
:1001B600B69BEECFB59BB9CFB49B9CCFB39B97CFE5
:0601C600B29BC4CF9CCFE8
:00000001FF
